:1000000000308A00FB280000223084000008031919
:10001000182801308D008C018C0B0C288D0B0B28BF
:100020004A308C008C0B122800000000800B09283D
:100030000034F830660006118614A801061406087C
:10004000F039A700061006140608F039A900A90E19
:100050002908A7040610A71F3228A80A2808633C0D
:1000600003181E28861008306600003406080F3971
:10007000A8002708F0392807860006140610A70EE6
:1000800006080F39A8002708F0392807860006144B
:1000900006100034192006112108A700362000346C
:1000A0000610061186101430A200042008306600E5
:1000B00030308600061406100530A2000420061415
:1000C000061031308C008C0B6328000000000614F1
:1000D000061019202030A1004A202830A1004A2013
:1000E0000830A1004A200C30A1004A200630A100AF
:1000F0004A200130A1004A200230A1004A200329F1
:10010000192006152608A700362000348C018D0121
:100110002108031022188C078C0C8D0CA2188C0758
:100120008C0C8D0C22198C078C0C8D0CA2198C0751
:100130008C0C8D0C221A8C078C0C8D0CA21A8C073F
:100140008C0C8D0C221B8C078C0C8D0CA21B8C072D
:100150008C0C8D0C003423088D0122020318B32867
:1001600022088C00BF288C010830A400A20D8C0D41
:1001700023080C0203188C008D0DA40BB628003444
:1001800010308C008F01A701A40CA30C031CCE28F7
:1001900025088F070318A70A2608A707A70C8F0CA6
:1001A0008E0C8D0C8C0BC428162B8D018E018C01AE
:1001B0008F012908031DDF2828080319F9281030AA
:1001C000AA000310A60DA70D8C0D8F0D29080F0294
:1001D000031DEC2828080C02031CF52828088C02B3
:1001E000031C8F0329088F0203148D0D8E0DAA0B9B
:1001F000E1280000003484011F3083050730831696
:100200008800831250284730A60080203430A60092
:1002100080204630A60080204F30A60080204E303F
:10022000A60080202030A60080205330A600802029
:100230005730A60080205230A60080202030A60033
:1002400080204230A60080207230A60080206930D5
:10025000A60080206430A60080206730A6008020A1
:100260006530A60080200430A100FA30A2000420EE
:10027000A10B35290230831688008312080838390B
:10028000C138880096019A0199018316811383125F
:10029000003086190130003A031D5C291908633CBF
:1002A000031C5B29990A1908643C031D5B299A0AFF
:1002B0000130A1004A205D29990100308D00080815
:1002C000C7390D04880006308C008C0B65290000AE
:1002D0000815081969290908970008308D000808D1
:1002E000C7390D04880006308C008C0B752900007E
:1002F000081508197929090898001708023C031CF9
:1003000089291808023C031C892917089500180838
:10031000940015089702140898021A080139003A47
:10032000031DDD2A16081802031CEE291808960082
:1003300016081D3C031CAD2917081D3C031CAD29E4
:10034000160D9200920D920DF8309205170D930044
:10035000930D930DF8309305EA2916083B3C031CD6
:10036000C02917083B3C031CC029160D9200920DB2
:10037000FC309205170D9300930DFC309305EA298C
:1003800016084F3C031CD72917084F3C031CD729DC
:100390001608A1000330A20086200D08920017085D
:1003A000A1000330A20086200D089300EA29160858
:1003B0007F3C031CE62917087F3C031CE629031039
:1003C000160D92000310170D9300EA2916089200EB
:1003D00017089300920E0F309205F7299208031D1B
:1003E00092039208031DF6299601F729960302301D
:1003F000A1004A204630A600802012080C3C0318B9
:10040000032A0C30920001309800120818020318D9
:100410000E2AFF30A6008020980A052A18080C3CF6
:10042000031C172A2030A6008020980A0E2A1608DE
:10043000633C03183F2A1608A2006430A300AB20D7
:1004400030300D07A200A60080201608A2000A3056
:10045000A300AB200D08A2000A30A300AB2030306F
:100460000C07A300A60080201608A2000A30A300F3
:10047000AB2030300C07A200A6008020682A960826
:1004800003195F2A2030A60080201608A2000A3037
:10049000A300AB200D08A2000A30A300AB2030302F
:1004A0000C07A300A60080201608A2000A30A300B3
:1004B000AB2030300C07A200A6008020682A203034
:1004C000A60080202030A60080202030A6008020BA
:1004D000C030A1004A205230A6008020930E0F3079
:1004E000930513080C3C0318772A0C309300013055
:1004F0009800130818020318822AFF30A6008020F3
:10050000980A792A18080C3C031C8B2A2030A60074
:100510008020980A822A1708633C0318B32A170818
:10052000A2006430A300AB2030300D07A200A6006B
:1005300080201708A2000A30A300AB200D08A200FB
:100540000A30A300AB2030300C07A300A6008020A7
:100550001708A2000A30A300AB2030300C07A2001D
:10056000A6008020DC2A97080319D32A2030A60091
:1005700080201708A2000A30A300AB200D08A200BB
:100580000A30A300AB2030300C07A300A600802067
:100590001708A2000A30A300AB2030300C07A200DD
:1005A000A6008020DC2A2030A60080202030A60073
:1005B00080202030A6008020E72B9C0118089B009B
:1005C0009E0117089D000230A1004A202030A6009D
:1005D00080202030A60080205330A6008020573095
:1005E000A60080205230A60080203A30A60080204D
:1005F0002030A60080201E081C02031CD22B031DE5
:10060000052B1B081D020318D22B1D081B07A10078
:100610001C08A2000318A20A1E08A2072208A400B0
:100620002108A300A6010A30A500C0280E08A300D7
:100630000D08A2001D081B028C001C088F001E085C
:10064000031C1E0F8F020C08A4000F08A5000E0843
:10065000A7000D08A6000F08A9000C08A800D520C7
:100660000E08A0000D089F00A008031D3B2B1F08CB
:10067000633C03188D2B2008A7001F08A600A901C2
:100680006430A800D5200E08A2000D08A10030306B
:100690000D07A3000E08A4000318A40A2308A6004F
:1006A00080202008A7001F08A600A9010A30A80082
:1006B000D5200E08A2000D08A1000E08A7000D0805
:1006C000A600A9010A30A800D5200C08A2000F0836
:1006D000A30030300C07A4000F08A5000318A50ADA
:1006E0002408A60080202E30A60080202008A70025
:1006F0001F08A600A9010A30A800D5200C08A100F7
:100700000F08A20030300C07A3000F08A400031844
:10071000A40A2308A6008020CB2B2030A60080202E
:100720002008A7001F08A600A9010A30A800D520AC
:100730000E08A2000D08A1000E08A7000D08A600D3
:10074000A9010A30A800D5200C08A2000F08A300B8
:1007500030300C07A4000F08A5000318A50A2408D0
:10076000A60080202E30A60080202008A7001F08A9
:10077000A600A9010A30A800D5200C08A1000F0886
:10078000A20030300C07A3000F08A4000318A40A2D
:100790002308A60080203A30A60080203130A60031
:1007A0008020E72B4930A60080204E30A600802014
:1007B0004630A60080202030A60080202030A600F1
:1007C00080202030A60080202030A60080204829EC
:0207D0006300C4
:02400E00FA3F77
:00000001FF
